 AutoWrap

 Timestamp is 559d99da (Thu Jul 09 00:44:58 2015)

 Preferred load address is 0000000180000000

 Start         Length     Name                   Class
 0001:00000000 00000030H .idata$5                CODE
 0001:00000030 00000228H .rdata                  CODE
 0001:00000260 00002353H .text                   CODE
 0001:000025b8 000002d8H .xdata                  CODE
 0001:00002890 00000014H .idata$2                CODE
 0001:000028a4 00000014H .idata$3                CODE
 0001:000028b8 00000030H .idata$4                CODE
 0001:000028e8 00000050H .idata$6                CODE
 0001:00002940 000000afH .edata                  CODE
 0002:00000000 00000000H .data                   DATA
 0002:00000000 00000aa4H .bss                    DATA
 0003:00000000 00000270H .pdata                  DATA
 0004:00000000 00000058H .rsrc$01                DATA
 0004:00000060 00000370H .rsrc$02                DATA

  Address         Publics by Value              Rva+Base               Lib:Object

 0000:00000000       ___safe_se_handler_count   0000000000000000     <absolute>
 0000:00000000       ___safe_se_handler_table   0000000000000000     <absolute>
 0000:00000000       __ImageBase                0000000180000000     <linker-defined>
 0001:00000000       __imp_lstrlenW             0000000180001000     kernel32:KERNEL32.dll
 0001:00000008       __imp_HeapFree             0000000180001008     kernel32:KERNEL32.dll
 0001:00000010       __imp_GetProcessHeap       0000000180001010     kernel32:KERNEL32.dll
 0001:00000018       __imp_HeapAlloc            0000000180001018     kernel32:KERNEL32.dll
 0001:00000020       __imp_lstrcpynW            0000000180001020     kernel32:KERNEL32.dll
 0001:00000028       \177KERNEL32_NULL_THUNK_DATA 0000000180001028     kernel32:KERNEL32.dll
 0001:00000030       MainGuid                   0000000180001030     AutoWrap.obj
 0001:00000040       MenuGuid                   0000000180001040     AutoWrap.obj
 0001:00000050       DialogGuid                 0000000180001050     AutoWrap.obj
 0001:00000060       ??_C@_1DE@BGKMIKPD@?$AAE?$AAu?$AAg?$AAe?$AAn?$AAe?$AA?5?$AAR?$AAo?$AAs?$AAh?$AAa?$AAl?$AA?5?$AA?$CG?$AA?5?$AAF?$AAa?$AAr?$AA?5?$AAG?$AAr?$AAo?$AAu?$AAp?$AA?$AA@ 0000000180001060     AutoWrap.obj
 0001:00000098       ??_C@_1DE@LDAHMEKD@?$AAA?$AAu?$AAt?$AAo?$AA?5?$AAw?$AAr?$AAa?$AAp?$AA?5?$AAf?$AAo?$AAr?$AA?5?$AAF?$AAa?$AAr?$AA?5?$AAM?$AAa?$AAn?$AAa?$AAg?$AAe?$AAr?$AA?$AA@ 0000000180001098     AutoWrap.obj
 0001:000000d0       ??_C@_1BC@NMCLCAKE@?$AAA?$AAu?$AAt?$AAo?$AAW?$AAr?$AAa?$AAp?$AA?$AA@ 00000001800010d0     AutoWrap.obj
 0001:000000e4       ??_C@_11LOCGONAA@?$AA?$AA@ 00000001800010e4     AutoWrap.obj
 0001:000000e8       ??_C@_1CC@MHEGACBP@?$AAE?$AAx?$AAc?$AAl?$AAu?$AAd?$AAe?$AAF?$AAi?$AAl?$AAe?$AAM?$AAa?$AAs?$AAk?$AAs?$AA?$AA@ 00000001800010e8     AutoWrap.obj
 0001:00000110       ??_C@_17ECHFBE@?$AA?$CK?$AA?4?$AA?$CK?$AA?$AA@ 0000000180001110     AutoWrap.obj
 0001:00000118       ??_C@_1BE@GBKLIJMP@?$AAF?$AAi?$AAl?$AAe?$AAM?$AAa?$AAs?$AAk?$AAs?$AA?$AA@ 0000000180001118     AutoWrap.obj
 0001:00000130       ??_C@_1BI@JMKBMFLI@?$AAR?$AAi?$AAg?$AAh?$AAt?$AAM?$AAa?$AAr?$AAg?$AAi?$AAn?$AA?$AA@ 0000000180001130     AutoWrap.obj
 0001:00000148       ??_C@_19BFPOADG@?$AAW?$AAr?$AAa?$AAp?$AA?$AA@ 0000000180001148     AutoWrap.obj
 0001:00000158       ??_7?$DialogItemBinding@UFarDialogItem@@@@6B@ 0000000180001158     AutoWrap.obj
 0001:00000170       ??_7?$DialogBuilderBase@UFarDialogItem@@@@6B@ 0000000180001170     AutoWrap.obj
 0001:000001b8       ??_7PluginEditFieldBinding@@6B@ 00000001800011b8     AutoWrap.obj
 0001:000001c8       ??_C@_15EFLNJKHH@?$AA?$CF?$AAu?$AA?$AA@ 00000001800011c8     AutoWrap.obj
 0001:000001d0       ??_7PluginIntEditFieldBinding@@6B@ 00000001800011d0     AutoWrap.obj
 0001:000001e0       ??_7PluginDialogBuilder@@6B@ 00000001800011e0     AutoWrap.obj
 0001:00000228       ??_7PluginCheckBoxBinding@@6B@ 0000000180001228     AutoWrap.obj
 0001:00000238       ??_7PluginRadioButtonBinding@@6B@ 0000000180001238     AutoWrap.obj
 0001:00000248       ??_7PluginUIntEditFieldBinding@@6B@ 0000000180001248     AutoWrap.obj
 0001:00000270       __chkstk                   0000000180001270 f   chkstk.obj
 0001:00000270       _alloca_probe              0000000180001270     chkstk.obj
 0001:000002c0       ?GetLangString@PluginDialogBuilder@@MEAAPEB_WH@Z 00000001800012c0 f i AutoWrap.obj
 0001:000002d0       GetGlobalInfoW             00000001800012d0 f   AutoWrap.obj
 0001:00000350       SetStartupInfoW            0000000180001350 f   AutoWrap.obj
 0001:00000550       GetPluginInfoW             0000000180001550 f   AutoWrap.obj
 0001:000005b0       ?GetCommaWord@@YAPEB_WPEB_WPEA_W@Z 00000001800015b0 f   AutoWrap.obj
 0001:000006a0       ?SaveValue@?$DialogItemBinding@UFarDialogItem@@@@UEAAXPEAUFarDialogItem@@H@Z 00000001800016a0 f i AutoWrap.obj
 0001:000006a0       ?InitDialogItem@?$DialogBuilderBase@UFarDialogItem@@@@MEAAXPEAUFarDialogItem@@PEB_W@Z 00000001800016a0 f i AutoWrap.obj
 0001:000006b0       ?TextWidth@?$DialogBuilderBase@UFarDialogItem@@@@MEAAHAEBUFarDialogItem@@@Z 00000001800016b0 f i AutoWrap.obj
 0001:000006c0       ?DoShowDialog@?$DialogBuilderBase@UFarDialogItem@@@@MEAA_JXZ 00000001800016c0 f i AutoWrap.obj
 0001:000006d0       ??1?$DialogBuilderBase@UFarDialogItem@@@@MEAA@XZ 00000001800016d0 f i AutoWrap.obj
 0001:00000750       ?AddUIntEditField@?$DialogBuilderBase@UFarDialogItem@@@@UEAAPEAUFarDialogItem@@PEAIH@Z 0000000180001750 f i AutoWrap.obj
 0001:00000750       ?GetLangString@?$DialogBuilderBase@UFarDialogItem@@@@MEAAPEB_WH@Z 0000000180001750 f i AutoWrap.obj
 0001:00000750       ?CreateCheckBoxBinding@?$DialogBuilderBase@UFarDialogItem@@@@MEAAPEAU?$DialogItemBinding@UFarDialogItem@@@@PEAHH@Z 0000000180001750 f i AutoWrap.obj
 0001:00000750       ?CreateRadioButtonBinding@?$DialogBuilderBase@UFarDialogItem@@@@MEAAPEAU?$DialogItemBinding@UFarDialogItem@@@@PEAH@Z 0000000180001750 f i AutoWrap.obj
 0001:00000750       ?AddIntEditField@?$DialogBuilderBase@UFarDialogItem@@@@UEAAPEAUFarDialogItem@@PEAHH@Z 0000000180001750 f i AutoWrap.obj
 0001:00000760       ??_E?$DialogBuilderBase@UFarDialogItem@@@@MEAAPEAXI@Z 0000000180001760 f i AutoWrap.obj
 0001:00000760       ??_G?$DialogBuilderBase@UFarDialogItem@@@@MEAAPEAXI@Z 0000000180001760 f i AutoWrap.obj
 0001:00000790       ?ReallocDialogItems@?$DialogBuilderBase@UFarDialogItem@@@@IEAAXXZ 0000000180001790 f i AutoWrap.obj
 0001:000008b0       ?ItemWidth@?$DialogBuilderBase@UFarDialogItem@@@@IEAA_JAEBUFarDialogItem@@@Z 00000001800018b0 f i AutoWrap.obj
 0001:00000950       ?SaveValues@?$DialogBuilderBase@UFarDialogItem@@@@IEAAXXZ 0000000180001950 f i AutoWrap.obj
 0001:000009f0       ?MaxTextWidth@?$DialogBuilderBase@UFarDialogItem@@@@IEAA_JXZ 00000001800019f0 f i AutoWrap.obj
 0001:00000b10       ?SaveValue@PluginEditFieldBinding@@UEAAXPEAUFarDialogItem@@H@Z 0000000180001b10 f i AutoWrap.obj
 0001:00000b50       ??0PluginIntEditFieldBinding@@QEAA@AEBUPluginStartupInfo@@PEAPEAXHPEAHH@Z 0000000180001b50 f i AutoWrap.obj
 0001:00000c10       ?SaveValue@PluginIntEditFieldBinding@@UEAAXPEAUFarDialogItem@@H@Z 0000000180001c10 f i AutoWrap.obj
 0001:00000c60       ?InitDialogItem@PluginDialogBuilder@@MEAAXPEAUFarDialogItem@@PEB_W@Z 0000000180001c60 f i AutoWrap.obj
 0001:00000c90       ?TextWidth@PluginDialogBuilder@@MEAAHAEBUFarDialogItem@@@Z 0000000180001c90 f i AutoWrap.obj
 0001:00000ca0       ?DoShowDialog@PluginDialogBuilder@@MEAA_JXZ 0000000180001ca0 f i AutoWrap.obj
 0001:00000d50       ?SaveValue@PluginCheckBoxBinding@@UEAAXPEAUFarDialogItem@@H@Z 0000000180001d50 f i AutoWrap.obj
 0001:00000db0       ?SaveValue@PluginRadioButtonBinding@@UEAAXPEAUFarDialogItem@@H@Z 0000000180001db0 f i AutoWrap.obj
 0001:00000e00       ??0PluginUIntEditFieldBinding@@QEAA@AEBUPluginStartupInfo@@PEAPEAXHPEAIH@Z 0000000180001e00 f i AutoWrap.obj
 0001:00000ec0       ?SaveValue@PluginUIntEditFieldBinding@@UEAAXPEAUFarDialogItem@@H@Z 0000000180001ec0 f i AutoWrap.obj
 0001:00000f10       ?CreateCheckBoxBinding@PluginDialogBuilder@@MEAAPEAU?$DialogItemBinding@UFarDialogItem@@@@PEAHH@Z 0000000180001f10 f i AutoWrap.obj
 0001:00000f90       ?CreateRadioButtonBinding@PluginDialogBuilder@@MEAAPEAU?$DialogItemBinding@UFarDialogItem@@@@PEAH@Z 0000000180001f90 f i AutoWrap.obj
 0001:00001000       ??_EPluginDialogBuilder@@UEAAPEAXI@Z 0000000180002000 f i AutoWrap.obj
 0001:00001000       ??_GPluginDialogBuilder@@UEAAPEAXI@Z 0000000180002000 f i AutoWrap.obj
 0001:00001050       ProcessEditorInputW        0000000180002050 f   AutoWrap.obj
 0001:000015a0       ?AddDialogItem@?$DialogBuilderBase@UFarDialogItem@@@@IEAAPEAUFarDialogItem@@W4FARDIALOGITEMTYPES@@PEB_W@Z 00000001800025a0 f i AutoWrap.obj
 0001:00001630       ?AddTextAfter@?$DialogBuilderBase@UFarDialogItem@@@@QEAAPEAUFarDialogItem@@PEAU2@PEB_WH@Z 0000000180002630 f i AutoWrap.obj
 0001:00001700       ?AddButtons@?$DialogBuilderBase@UFarDialogItem@@@@QEAAXHPEBHHH@Z 0000000180002700 f i AutoWrap.obj
 0001:00001850       ?UpdateBorderSize@?$DialogBuilderBase@UFarDialogItem@@@@IEAAXXZ 0000000180002850 f i AutoWrap.obj
 0001:00001910       ??_GPluginIntEditFieldBinding@@UEAAPEAXI@Z 0000000180002910 f i AutoWrap.obj
 0001:00001910       ??_GPluginUIntEditFieldBinding@@UEAAPEAXI@Z 0000000180002910 f i AutoWrap.obj
 0001:00001910       ??_EPluginEditFieldBinding@@UEAAPEAXI@Z 0000000180002910 f i AutoWrap.obj
 0001:00001910       ??_EPluginRadioButtonBinding@@UEAAPEAXI@Z 0000000180002910 f i AutoWrap.obj
 0001:00001910       ??_GPluginRadioButtonBinding@@UEAAPEAXI@Z 0000000180002910 f i AutoWrap.obj
 0001:00001910       ??_G?$DialogItemBinding@UFarDialogItem@@@@UEAAPEAXI@Z 0000000180002910 f i AutoWrap.obj
 0001:00001910       ??_EPluginCheckBoxBinding@@UEAAPEAXI@Z 0000000180002910 f i AutoWrap.obj
 0001:00001910       ??_GPluginCheckBoxBinding@@UEAAPEAXI@Z 0000000180002910 f i AutoWrap.obj
 0001:00001910       ??_E?$DialogItemBinding@UFarDialogItem@@@@UEAAPEAXI@Z 0000000180002910 f i AutoWrap.obj
 0001:00001910       ??_EPluginIntEditFieldBinding@@UEAAPEAXI@Z 0000000180002910 f i AutoWrap.obj
 0001:00001910       ??_EPluginUIntEditFieldBinding@@UEAAPEAXI@Z 0000000180002910 f i AutoWrap.obj
 0001:00001910       ??_GPluginEditFieldBinding@@UEAAPEAXI@Z 0000000180002910 f i AutoWrap.obj
 0001:00001940       ?AddIntEditField@PluginDialogBuilder@@UEAAPEAUFarDialogItem@@PEAHH@Z 0000000180002940 f i AutoWrap.obj
 0001:00001a50       ?AddUIntEditField@PluginDialogBuilder@@UEAAPEAUFarDialogItem@@PEAIH@Z 0000000180002a50 f i AutoWrap.obj
 0001:00001b60       OpenW                      0000000180002b60 f   AutoWrap.obj
 0001:000024a0       memcpy                     00000001800034a0 f   libCRT64:memcpy.obj
 0001:000024d0       wcschr                     00000001800034d0 f   libCRT64:strchr.obj
 0001:000024f0       ??_V@YAXPEAX@Z             00000001800034f0 f   libCRT64:delete_array.obj
 0001:00002500       ??3@YAXPEAX@Z              0000000180003500 f   libCRT64:delete.obj
 0001:00002510       ??_U@YAPEAX_K@Z            0000000180003510 f   libCRT64:new_array.obj
 0001:00002520       memset                     0000000180003520 f   libCRT64:memset.obj
 0001:00002550       ??2@YAPEAX_K@Z             0000000180003550 f   libCRT64:new.obj
 0001:00002560       free                       0000000180003560 f   libCRT64:free.obj
 0001:00002590       malloc                     0000000180003590 f   libCRT64:malloc.obj
 0001:00002890       __IMPORT_DESCRIPTOR_KERNEL32 0000000180003890     kernel32:KERNEL32.dll
 0001:000028a4       __NULL_IMPORT_DESCRIPTOR   00000001800038a4     kernel32:KERNEL32.dll
 0002:00000290       ?Opt@@3UOptions@@A         0000000180004290     AutoWrap.obj

 entry point at        0000:00000000

 Static symbols

